:020000040000FA
:1000000000004F3094001E28831A0D281710950009
:10001000030E960004089800A12883121714950077
:10002000030E960004089800A12818088400160EF4
:100030008300950E150E17188316090014308400DE
:100040003B309100840A8001910B2228372805302B
:10005000030503190800053C080014078400312833
:10006000840000088D00840A00088E000800133008
:100070009E008A01830177289E0B422813309E0040
:1000800043205D2008009F08031D4A280618080029
:10009000B2305A289F1B4E289F030800061C532885
:1000A00003309F0008001F037F399F009F17031D27
:1000B0000800B2309F009D140800A008031D6428AA
:1000C00086180800B2307428A01B6828A003080016
:1000D000861C6D280330A000080020037F39A00093
:1000E000A017031D0800B230A0001D1408008316DD
:1000F0007F308105C0308105013081048312810188
:100100009D01FF308604FB308B058316F330860596
:100110008312F7308605FB308605A52080308B04DE
:100120001D1C9528FE309D05D5200B1D9A28FB30FF
:100130008B053C209D1C9F28FD309D05DB20A720C2
:100140009028A3281528A2280800A1010800023041
:1001500099009A01E1202208FF3EA20032302202DB
:1001600027200319B5280230A100323022022202D2
:100170000230A1008D050D080319BF28A10101302F
:1001800022020318C5280130A200A1010A3086040A
:100190000130A10004308604FB3086050230A10046
:1001A00008308604F730860508000130A1000800F9
:1001B000FA30A20008000230A10008000130A100BE
:1001C000080001302D20840AE7208A0108000D086C
:1001D0000E04031908000130FA205430F4208D0376
:1001E0000D0FE7288E03E728000000008F008F0B1B
:1001F000F72808009000F030F620900BFB2808004C
:00000001FF
